:1000000019C08CC0189518951895189518951895BD
:100010001895189518951895189518951895189578
:100020001895189518951895189518951895189568
:10003000189518958FEF8DBFC0EEE0EE4E2E84E040
:100040008EBFD4E0F4E05F2EEEEFF3E0A0E0B1E08D
:1000500088278D933197E9F767D4662488E78AB9B2
:1000600086E887B980E08BB980E088B95A9A5E9AB1
:10007000789480E080930A013DD48CE09DD4E6E43E
:10008000FBE030D4E1E0F0E046D432D4E6E5FBE03A
:1000900029D484EF91E0BCD4ECE5FBE023D484EFD9
:1000A00091E0B6D4E2E6FBE01DD48AEF90E0B0D454
:1000B000E4E6FBE017D48AEF90E0AAD4E6E6FBE0A2
:1000C00011D48AEF90E0A4D4E8E6FBE00BD48AEFE9
:1000D00090E09ED4EAE6FBE005D48AEF90E098D465
:1000E000ECE6FBE0FFD38AEF90E092D4EEE6FBE093
:1000F000F9D38AEF90E08CD4E0E7FBE0F3D3E3E0C0
:10010000F0E009D4F7D3E2E7FBE0ECD38DB38160F4
:100110008DBB85E083BF8895F6CFABCF0F921F9242
:100120002F923F924F925F927F92AF92BF920F9326
:100130001F932F933F934F935F936F937F938F936F
:100140009F93AF93BF93CF93DF93EF93FF938FB7BB
:100150008F938DB38E7F8DBB84E690E059D40027BA
:10016000BB27A6E28C9184FB0EF401E040E004176B
:1001700009F001C01CD10027BB27A9E28C9182FBAA
:100180000EF401E040E0041709F02BC05E9888E20D
:1001900090E03ED4419A429A8AE090E039D4429865
:1001A0008AE090E035D44198429A8AE090E030D4D9
:1001B00042980027BB27A9E28C9187FB0EF401E04F
:1001C00040E0041709F001C029D00027BB27A9E2AD
:1001D0008C9187FB0EF401E041E0041709F001C0A7
:1001E00045D18F918FBFFF91EF91DF91CF91BF915B
:1001F000AF919F918F917F916F915F914F913F91BF
:100200002F911F910F91BF90AF907F905F904F9073
:100210003F902F901F900F90189508956BD38FE704
:1002200011E077D3E2E8FBE05DD380E08093090141
:100230000027BB27A6E28C9180FB0EF401E040E092
:10024000041709F005C0A9E0B1E08C918F5F8C9391
:100250000027BB27A9E28C9181FB0EF401E040E06E
:10026000041709F005C0A9E0B1E08C918E5F8C9372
:100270000027BB27A9E28C9180FB0EF401E040E04F
:10028000041709F005C0A9E0B1E08C918C5F8C9354
:100290000027BB27A6E28C9185FB0EF401E040E02D
:1002A000041709F005C0A9E0B1E08C91885F8C9338
:1002B000009109010A3008F003C0E4E6FBE012D324
:1002C000A8ECB4E0E9E0F1E0D3D304D311D381E0AA
:1002D00080930101009101010F3010F009F04AC034
:1002E00080E08093000180E0809302010091020190
:1002F000073010F009F01FC0A0E0B1E00C9142E01F
:10030000049F0C9200910001BB27A6E28C9183FB15
:10031000882780F9482F040FA0E0B1E00C93429A9F
:100320008AE090E075D34298A2E0B1E08C918F5FB3
:100330008C9308F4DBCF009109014FE0049FA3E008
:10034000B1E00C920091030140910101040FA3E080
:10035000B1E00C93A3E0B1E0EC91FF27A0E0B1E0A5
:1003600091E07BE7D8D3A1E0B1E08C918F5F8C93D3
:1003700008F4B0CF84E690E04BD35E9A8AEF809386
:10038000040181E080930601B3D2E0E9FBE0AAD248
:100390007BD20027BB27A9E28C9182FB0EF401E0FF
:1003A00040E0041709F001C0F4CFA4D20895A2D20E
:1003B000EEE9FBE097D29CD2E6E4FBE093D2002783
:1003C000BB27A6E28C9184FB0EF401E041E0041708
:1003D00009F001C04AC081E08093010181E090E012
:1003E000A7E0B1E08D939C93A7E0B1E00D911C9143
:1003F0000A3F50E0150710F009F00EC0A7E0B1E089
:10040000ED91FC91A1E0B1E091E07BE784D3A7E01E
:10041000B1E059D208F4E8CF5E9A8AEF80930401E4
:1004200082E08093060166D2E6E4FBE05BD260D214
:10043000ECEAFBE057D228D20027BB27A9E28C9137
:1004400082FB0EF401E040E0041709F001C0F4CF94
:100450000027BB27A6E28C9184FB0EF401E040E06C
:10046000041709F001C0E8DF45D2089543D28FE7B1
:1004700011E04FD2ECEBFBE035D23AD2E6E4FBE000
:1004800031D2E1E0F0E047D281E0809301010091B8
:1004900001010F3010F009F0A8C180E08093000145
:1004A00080E08093020100910201073010F009F012
:1004B0001CC0A0E0B1E00C9142E0049F0C920091BE
:1004C0000001BB27A6E28C9183FB882780F9482F87
:1004D000040FA0E0B1E00C93429A4298A2E0B1E090
:1004E0008C918F5F8C9308F4DECFA1E0B1E0EC91AA
:1004F000FF27A5E0B1E091E01FD3409105010091F5
:100500000001041709F401C001C068C10091010194
:100510004FE0040FA3E0B1E00C93A3E0B1E0EC9155
:10052000FF27A5E0B1E091E007D3409105010091DC
:100530000001041709F401C001C050C1009101017C
:100540004EE1040FA3E0B1E00C93A3E0B1E0EC9125
:10055000FF27A5E0B1E091E0EFD2409105010091C5
:100560000001041709F401C001C038C10091010164
:100570004DE2040FA3E0B1E00C93A3E0B1E0EC91F5
:10058000FF27A5E0B1E091E0D7D2409105010091AD
:100590000001041709F401C001C020C1009101014C
:1005A0004CE3040FA3E0B1E00C93A3E0B1E0EC91C5
:1005B000FF27A5E0B1E091E0BFD240910501009195
:1005C0000001041709F401C001C008C10091010134
:1005D0004BE4040FA3E0B1E00C93A3E0B1E0EC9195
:1005E000FF27A5E0B1E091E0A7D24091050100917D
:1005F0000001041709F401C001C0F0C0009101011D
:100600004AE5040FA3E0B1E00C93A3E0B1E0EC9164
:10061000FF27A5E0B1E091E08FD240910501009164
:100620000001041709F401C001C0D8C00091010104
:1006300049E6040FA3E0B1E00C93A3E0B1E0EC9134
:10064000FF27A5E0B1E091E077D24091050100914C
:100650000001041709F401C001C0C0C000910101EC
:1006600048E7040FA3E0B1E00C93A3E0B1E0EC9104
:10067000FF27A5E0B1E091E05FD240910501009134
:100680000001041709F401C001C0A8C000910101D4
:1006900047E8040FA3E0B1E00C93A3E0B1E0EC91D4
:1006A000FF27A5E0B1E091E047D24091050100911C
:1006B0000001041709F401C001C090C000910101BC
:1006C00046E9040FA3E0B1E00C93A3E0B1E0EC91A4
:1006D000FF27A5E0B1E091E02FD240910501009104
:1006E0000001041709F401C001C078C000910101A4
:1006F00045EA040FA3E0B1E00C93A3E0B1E0EC9174
:10070000FF27A5E0B1E091E017D2409105010091EB
:100710000001041709F401C001C060C0009101018B
:1007200044EB040FA3E0B1E00C93A3E0B1E0EC9143
:10073000FF27A5E0B1E091E0FFD1409105010091D4
:100740000001041709F401C001C048C00091010173
:1007500043EC040FA3E0B1E00C93A3E0B1E0EC9113
:10076000FF27A5E0B1E091E0E7D1409105010091BC
:100770000001041709F401C001C030C0009101015B
:1007800042ED040FA3E0B1E00C93A3E0B1E0EC91E3
:10079000FF27A5E0B1E091E0CFD1409105010091A4
:1007A0000001041709F401C001C018C00091010143
:1007B00041EE040FA3E0B1E00C93A3E0B1E0EC91B3
:1007C000FF27A5E0B1E091E0B7D14091050100918C
:1007D0000001041709F401C036C000C0A1E0B1E077
:1007E0008C918F5F8C9308F452CE84D081D0EAEC48
:1007F000FBE078D05E9A8AEF8093040181E08093D9
:10080000060142D00027BB27A9E28C9182FB0EF49F
:1008100001E040E0041709F001C0F4CF6BD0E6E43A
:10082000FBE060D065D0ECEDFBE05CD0E1E0F0E017
:1008300072D05C9AE2E0F0E06ED05C98E1E0F0E02B
:100840006AD058D0089556D0EAEEFBE04BD050D095
:10085000E6E4FBE047D05E9A8AE58093040189E0F4
:100860008093060111D00027BB27A9E28C9182FB5F
:100870000EF401E040E0041709F001C0F4CFE2E01B
:10088000F0E049D037D0089580E080930101409195
:10089000060100910101041710F009F013C05B9AE2
:1008A000A4E0B1E08C919927B3D05B98A4E0B1E0CB
:1008B0008C919927ADD0A1E0B1E08C918F5F8C93A2
:1008C00008F4E5CF0895ED91FC91EF5FFF4FFC93A5
:1008D000EE930895A8ECB4E08D91882311F066D0D2
:1008E000FBCF0895A4D0802D11F060D0FBCF0895E8
:1008F00080EC62C081E060D014D080E85DC08FE7FA
:10090000213039F08FEB223021F08FE8233009F0CD
:100910008FEC810F51C088EE93E07AD03197D9F7F0
:10092000089583E0992774C08AEF90E071D0259AEA
:10093000249A239A229A219A209A289885E090E076
:1009400067D029982D982C982B9A2A9A299AEF9358
:10095000FF93E5E1F0E050D0FF91EF91299855D059
:10096000299AEF93FF93E5E1F0E046D0FF91EF91F4
:1009700029984BD0299AEF93FF93E5E1F0E03CD022
:10098000FF91EF91299841D02A98299AEF93FF93EC
:10099000E5E1F0E031D0FF91EF91299836D088E27F
:1009A0000BD08EE009D086E007D00895289A829572
:1009B00005D004D02AD008952898F9CF859510F451
:1009C0002A9A01C02A98859510F42B9A01C02B9879
:1009D000859510F42C9A01C02C98859510F42D9AC9
:1009E00001C02D98299AEF93FF93E5E1F0E004D040
:1009F000FF91EF91299808953197F1F70895689440
:100A000062F80895E89462F8089581E090E000C0EB
:100A1000EF93FF93EE27E82BE92B31F0EAEFF0E0BC
:100A20003197F1F70197D1F7FF91EF910895C895AC
:100A3000319600200895000F111F221F331F0895C3
:100A400000951095209530950F5F1F4F2F4F3F4F0A
:100A50000895019110810EC0019111912191308171
:100A60000BC00191108117FF05C03FEF2FEF04C0AD
:100A7000008111272227332737FF03C0E1DF8DE2F2
:100A80008D93CF93DF93CF92DF92EF92AA24BB2472
:100A9000CC24DD24EE2440E2CAE0DD2755E093E3D8
:100AA0008881890F87FD9F7083FD907F891B8993C3
:100AB0005A95A9F7C0DFAA1CBB1CCC1CDD1CEE1C80
:100AC0004A9551F7E894EFE0FF2782910ED0EB3082
:100AD000E0F71EF068948A2D0CD088278D93EF9054
:100AE000DF90CF90DF91CF910895982F829501D01C
:100AF000892F8F70805D26F0803309F40895689403
:100B00008D930895F999FECFE1BDF2BD3196089518
:100B100091E001C092E07B3751F47FB7F894F2DFA7
:100B20008D9180BDFA9AF99A9A95C9F77FBF772778
:100B3000089591E001C092E0E5DFF89A80B58D93C9
:100B40009A95D1F708955757572E4156522E344D46
:100B5000472E434F4D0047534D3A00002B33383654
:100B6000000034003000380033003200310037001C
:100B700039002020496E73657274204361726420CD
:100B8000200043617264206E756D6265723A0000E8
:100B900043617264207772697474656E00004572F7
:100BA0006173696E67204361726473002020204383
:100BB0006172647320657261736564002020202077
:100BC000436865636B696E6700002043617264204F
:100BD0006578636570746564202000002020202003
:100BE000556E6C6F636B656400002020204361725A
:080BF000642077726F6E67004C
:00000001FF
